:100000000EC077C080C011C010C00FC00EC00DC0A0
:100010000CC00BC00AC009C008C007C006C011242C
:100020001FBECFEDCDBF2BD078C0EACFA89584B747
:10003000877F84BF88E10FB6F89481BD11BC0FBEE5
:1000400087B3886187BBC19AC29AA99A85B785BFD1
:100050008BB780668BBF94E080E80FB6F89486BDBE
:1000600096BD0FBE0895B19902C08FEF089580E04C
:100070000895B29902C08FEF089580E008951F930C
:10008000D5DF789485B7877E806185BF10E085B71E
:10009000806285BF889585B78F7D85BFE4DF882323
:1000A00089F0109519F088B3886102C088B3877E03
:1000B00088BB83EC99E00197F1F700C00000D3DF23
:1000C0008823E9F7D6DF882359F0112319F088B384
:1000D000877E02C088B3886188BBCBDF8823E9F7BD
:1000E000112319F088B3886102C088B3877E88BB6A
:1000F000CECF1F920F920FB60F9211240F900FBE0A
:100100000F901F9018951F920F920FB60F92112407
:0E0110000F900FBE0F901F901895F894FFCF20
:00000001FF
